:020000040000FA
:0600000008308A00002810
:08000800FC00030EFD000408DA
:10001000FF000A08FE008312031309308A002B290F
:100020007E088A007F0884007D0E8300FC0E7C0E13
:020030000900C5
:020040000000BE
:100C0000EE24F434E1346936693D67372E17001756
:100C10000000682AA0326537773AF237A035F03005
:100C20006538F230A0396F3A6210A0326932E33988
:100C3000EE376537F431E43260176C28E132E5397C
:100C400063106534EB317910F5372039F4326534AF
:100C50006E39F4326310EE376537F431EF342E37E6
:100C60000000682AA0326537773AF237A035F334AE
:100C70006E10F7376310EE376537F431E432001742
:100C80000000692867377410F03CBD320000731013
:100C9000F132801E00006C10EE32801E00006630C3
:100CA0006F39BA3600100000E1216E37F437631057
:100CB000EE376537F4317410A037683AA032EC296A
:100CC000ED34E5297639F23220172010201020105B
:100CD000F32461107310F232653B203975396E3799
:100CE000EE34A033F43000100000A01F00006F2687
:100CF000EB37EE34A0336F332039A0304822D021B7
:100D00007310F232653B2E392E1700006F26EB3739
:100D1000EE34A0336F332039EC29ED345310F23226
:100D2000653B2E392E1700002010201020102010B7
:100D300020105710EC32EF31E5365410A037CC2993
:100D4000CD243328203020102010201020107710C0
:100D5000F73B73176936E436F632E334F332631740
:100D6000ED3720102010201020102E1980190000BF
:100D7000EF2BEC3A2032EF3CA03A6936E53574109F
:100D8000A037E539203AF03A7410653470106136B6
:100D9000E53C3F3900004E30AC3770106F39E5311B
:100DA000E4327710F4342034F439F230753A2038D4
:100DB0002010201020102010201020102010003FA4
:100DC00000005930F3322016EF337410A037E539A4
:100DD000753A2038E5367537201020102010201085
:100DE00020102010201020102010003F0000F32AB7
:100DF000A032683AA032D02AC417D7272027F23071
:100E00006F39A03B7531743AEE37A0396F3A6310F1
:100E10006F34F337AC327530E539741065345210E5
:100E2000C724542461107239F7376210F43A6F3ACC
:100E300020376F3A6D10F637A032EE3700170000FA
:100E40006C28E132E53963106F34F337A032A030FB
:100E5000EF316637E734F23AF430EF342037E536D5
:100E6000683AE437001D00004330ED376C38F43247
:100E7000EC32A03CF5306F3AE136693AA0314414C7
:100E8000432420282013EC29ED345022A0142010F4
:100E9000003F000053306538E93179337310F23286
:100EA000653B2039E1367537EC3079362810482219
:100EB000D0216F106C37A93C20102010003F00009B
:100EC00045307437F2326510653B7939683AEE3453
:100ED000A033E1367537EC3079362810F429F43038
:100EE000E33449107328A014003F0000EF21663757
:100EF000E734F23AF430EF3420376134A039653109
:100F0000EE326310EE30E5316C36E432001700004B
:100F1000E82BF4306910A039F93649102028E43064
:100F20007232F332A0397414653470106136E53CC6
:100F30002939E01F000065276D3AF330BF352810CE
:100F4000F32AE13A6C36A03C3519AE1A3519AE1ABF
:100F50003519AE1A3018291800300000E123653A1F
:100F6000E13BBF3C2810D024611064326539F3396D
:100F70006F102033EF3CF23A7210F537653A293999
:100F800000300000D024611064326539F3396F10ED
:100F90002033683AA032EC29ED34E5297639F23273
:100FA000E01F0000E529753A2038F3346310ED376F
:100FB0006C38F432AE3250306539F3394C10C622F9
:100FC000202A6F3A6710A0376131EB31201649298A
:100FD000C823202A6F3A6510693C2E3A0000652923
:0C0FE000E539743AEE34AE332E170000F1
:101000000428FF34FF34FF3403138316FF309F009E
:101010000516881708160814831217308A001A2735
:1010200008308A0018308A00492008308A00A5015B
:101030009E2392200030AE20202211308A00802191
:1010400008308A0014308A005D2408308A009D210F
:101050001D21922018308A00032008308A000918C8
:10106000CC23A51D382816308A006D2608308A004A
:10107000BC2217308A00502708308A0016308A00B8
:10108000602608308A00AF1F2F2808308A00002809
:1010A0000F39820730343134323433343434353408
:1010B00036343734383439344134423443344434A8
:1010C0004534463408308A002108F039A70003105F
:1010D000A70CA70CA70C270C5020842021080F393F
:1010E00050208420080002307620080085128316E4
:1010F0008601831286000000000088150000881118
:1011000083168603831208008516831686018312D0
:1011100086000000000088150000881183168603F1
:101120008312080083168811051685128312FF307A
:10113000EF203C3076200530EF200C307620053053
:10114000EF20063076200530EF2001307620023087
:10115000EF20023076200530EF200800AE00063088
:10116000AD004B21AC0DAB0DAC0C2B0803190800E6
:10117000603C031DBE28C0307620C0282B08842088
:101180002C0803190800603C031DC928C0307620D4
:10119000CB282C088420AE0FB128AD0AB128C0306E
:1011A0007620080050208420080008308A0064302F
:1011B0004B242208502084200A304B24220850203F
:1011C00084202008502084200800831603179000F4
:1011D00000000000900BE828831203130800831618
:1011E00003179100F930E520F930E520F930E520CA
:1011F000F730E52083160317910BF22883120313AF
:1012000008001030EF2008001030A300FA30EF2063
:10121000A30B06290800831603179200FA30EF206B
:10122000FA30EF20FA30EF20FA30EF208316031760
:10123000920B0E2983120313080031309000C03046
:101240008B000C1083160C14831603179301940162
:101250008312031308000C1083160317940F31290F
:10126000930A1408831203130F39031D3829A51597
:10127000A40B3C29A517A516251E4329FF30A40061
:10128000A51E432925172512AF1600308A00102805
:101290008312031308002D0803178F0003132E0871
:1012A00003178D0083168C170C14000000008312A6
:1012B0000E080313AB0003170C080313AC0008005F
:1012C00003178D008F0183168C130C1483120C08E6
:1012D0000313A300080083120313210803178C00D3
:1012E00083120313200803178D0083168C130C152B
:1012F00055308D00AA308D008C14000000008C1831
:101300007F2903130D128312080083168814831299
:1013100008008316881083128810080083160815A9
:101320008312080083160811831208110800083080
:10133000E5280317800D0313080085218E2108007E
:1013400085218E21881CA229081DA429972192217C
:1013500097218921972108008921922197218521B0
:1013600097218E21972108008521881CB529972176
:1013700003100819031489218E2197210800B42134
:1013800099210800BF21BF21BF21BF21BF21BF215B
:10139000BF21BF21080099218E21031C9221972192
:1013A000B4210800A00020308400CB21CB21CB2128
:1013B000CB21CB21CB21CB21CB21E22108008E21D7
:1013C000B42108009221B4218E21080083168601E1
:1013D00083122E0886000A301C222D0886000B304E
:1013E0001C222C0886000C301C222B0886000D3095
:1013F0001C2208008316860183122E0886000A30FC
:101400001C222D0886000B301C22831686018603C1
:1014100083120C301022AC000D301022AB000800FB
:101420008500081300000608081708008500081347
:101430008717871308170800850088128816080088
:1014400083168501860108138812831208178816EF
:1014500085011430EF20A0224922AF010800AF120D
:101460003430AE000130AD00FA212C08A300AF19D2
:10147000412AA31B0800251692200930AE20AF1583
:101480000800A31F0800251692203130AE20AF11AE
:1014900008001230AE000130AD000030AC0000306A
:1014A000AB00E6211830AE000130AD000030AC00DA
:1014B0000030AB00E6210230AE000130AD0000305C
:1014C000AC000130AB00E6210430AE000130AD00CD
:1014D0000030AC000D30AB00E6210630AE0001302C
:1014E000AD00C030AC008F30AB00E6215830AE000C
:1014F0000130AD00E0306021AC00E1306021AB0094
:10150000E6215A30AE000130AD00E2306021AC007F
:10151000E3306021AB00E6215C30AE000130AD006D
:10152000E4306021AC00E5306021AB00E6211230F0
:10153000AE000130AD00FA212C17AC17E6210800EF
:101540001430AE000130AD004030AC000030AB00D4
:10155000E6210130EF201430AE000130AD00FA2159
:101560002C1BA92A3630AE000130AD00FA21AC1B8D
:101570000800A00BA02AA92AAF1A2F2283168601E1
:10158000860383120918CC2308301022AC000930DE
:101590001022AB002C080319080004302C02031998
:1015A000D62A08302C020319D822BE2AD922BE2AF4
:1015B0000800831686018603831201301022003052
:1015C000102201301022B600B000AB000030102213
:1015D000B700B100AC002F133C30A70038308400B6
:1015E0000918CC23003010228000840A0130102218
:1015F0008000840AA703A70BF02A2F1408304402A6
:10160000031D062B063045020319982D08304402AD
:10161000031D0800450803195E2E08000230AE00C5
:101620000130AD00FA214030AC04E6210800A030C2
:1016300084003C303702A700B200403C0318222B44
:101640004030A7003208031908000030102283162A
:1016500080008312840AA70B2F2B80010800013021
:101660001022831680008312840AA70B252B080002
:101670000918CC23831686018312C03086000430FB
:101680001C220030860005301C22370886000630F8
:101690001C223608860007301C222F163830AE0078
:1016A0000130AD00FA212B1C08002F128316860191
:1016B0008312383084003C30A7000918CC2300087E
:1016C000860000301C22840A0008860001301C229B
:1016D000840AA703A70B5D2B320803190800A70093
:1016E000A03084000008860000301C22840AA70B6A
:1016F0007A2B822B0008860001301C22840AA70B5B
:10170000722B08000030860001301C22080083166E
:10171000860183122B08860000301C222C088600CC
:1017200001301C2208002F1B992B003010222F178C
:101730009C2B013010222F13AC00080003179101DD
:1017400093019401950196019701492CCE01CF0197
:101750005030D000D1013230EF20091CB52B1830A9
:101760008A009B200B308A00A62B03130130CE0287
:101770000318C42BCF020318C42BD0020318C42BA8
:10178000D1020318C42B9E2B03130918CC23031773
:10179000111DB52B9101492C03171119492C8316E2
:1017A00003130608831203179900831203131830DA
:1017B0008A009B200B308A008312031719088316B6
:1017C00003138600831203132208031792001118D3
:1017D0000C2C1208503C03180B2C9E2303171114D9
:1017E000120898001208453C0318FA2B1208633CB3
:1017F0000318072C12089E3C0318022C1208BC3C4C
:101800000318042C0130052C02309A00492C0230B8
:101810009A001115492C9E2B02301A020319212C13
:101820001208013C0318182C12081F3C0318332C13
:101830001208233C0318202C1208413C0318352CB5
:10184000312C1208013C0318292C12081F3C0318E4
:10185000332C1208273C0318312C1208453C03187E
:10186000352C9101E92B9213362C9217920D940D81
:10187000950D960D970D930A103092001A08023CB0
:10188000031D442C2030920013081202031D492C22
:10189000111503130800A100A2012108A002031CD6
:1018A000532CA20A4D2CA00722080800840A000825
:1018B000A807031C5E2CA90F5E2CAA0A840300084B
:1018C000A9070318AA0A0800A807031C0800A90F03
:1018D0000800AA0A08002708AC020318732C01307C
:1018E000AB02031C792C2608AB02031C792C0314D1
:1018F0000800031008008400A801A901AA0100083B
:10190000AB00840A0008840AA807031C8B2C013052
:10191000A9070318AA0A2B08A9070318AA0A023064
:10192000B1020318972C0130B002031C9D2C310822
:10193000031D7F2C3008031D7F2C2F1DA82C32087F
:101940000319A82CB100B0012F11A03084007F2C06
:101950002A08A8070318A90A2809AC002909AB001E
:101960000800E0306021BE00E1306021BF00E230BD
:101970006021C000E3306021C100E4306021C2007A
:10198000E5306021C3000800E0306021EE00E13066
:101990006021EF00E2306021F000E3306021F100CF
:1019A000E4306021F200E5306021F30008004E08C9
:1019B000D8004F08D9005008DA005108DB0052085F
:1019C000DC005308DD00E0306021CE00E130602112
:1019D000CF00E2306021D000E3306021D100E4305C
:1019E0006021D200E5306021D3005408DE005508A4
:1019F000DF005608E0005708E10000306021D40005
:101A000001306021D50002306021D6000330602112
:101A1000D70008003E08B8003F08B9004008BA00E7
:101A20004108BB004208BC004308BD00E030602113
:101A3000BE00E1306021BF00E2306021C000E33031
:101A40006021C100E4306021C200E5306021C300A4
:101A50000800FF30B800B900BA00BB00BC00BD00F0
:101A60000800D7240A252925D801D901DA01DB018C
:101A7000DC01DD010830C4000630C500C6010130BC
:101A8000C7000830C800C9010630CA000430CB00C6
:101A9000CC010130CD000030B6002A30B70025114E
:101AA00008306021A00000306021A00604306021D1
:101AB000A005031D8A2D09306021A000013060219E
:101AC000A00605306021A005031D8A2D0A30602183
:101AD000A00002306021A00606306021A005031D91
:101AE0008A2D0B306021A00003306021A006073052
:101AF0006021A005031D8A2D08306021DE00093019
:101B00006021DF000A306021E0000B306021E1003D
:101B1000382308000C306021DE000D306021DF002A
:101B20000E306021E0000F306021E1003823080012
:101B3000251C080001304702031D08000830480238
:101B4000031D080000304902031D080006304A0248
:101B5000031D080004304B02031D080001304D0234
:101B6000031DCB2D003060215E02031D08000130F3
:101B700060215F02031D0800023060216002031D26
:101B80000800033060216102031D08000A25CD0A08
:101B9000D724382308002519080083171E30840035
:101BA0004E088000840A4F088000840A5008800094
:101BB000840A51088000840A52088000840A53086D
:101BC0008000831325152A2708005208D6005308E1
:101BD000D7005408D8005508D90000306021D20041
:101BE00001306021D30002306021D4000330602135
:101BF000D50008000918CC23251D080010306021ED
:101C0000DA0011306021DB0012306021DC0013307B
:101C10006021DD0008306021D60009306021D70046
:101C20000A306021D8000B306021D90083171E30A4
:101C300084000008B800840A0008B900840A00087B
:101C4000BA00840A0008BB00840A0008BC00840AA9
:101C50000008BD008313B124ED25C424DC26091837
:101C6000CC234530C600C7015E08C8005F08C90024
:101C70001430C9070318C80A0317A50F402EA40A79
:101C800024080313CA00031725080313CB00CC0153
:101C9000CD014030CE001130CF00CF260918CC2323
:101CA0000830C400C5014808B6004908B7000E3026
:101CB000B7070318B60A0918CC23382B0918CC2308
:101CC00001304F02031D7B2E003060215602031DA0
:101CD0000800013060215702031D08000230602116
:101CE0005802031D0800033060215902031D08003B
:101CF00013308A009B2B11304F020319802E0800ED
:101D0000113060215D02031D062F103060215C023E
:101D1000031D062F003060215602031D080001300C
:101D200060215702031D0800023060215802031D84
:101D30000800033060215902031D0800A51CB42EC1
:101D4000083060215202031D08000930602153024F
:101D5000031D08000A3060215402031D08000B30E7
:101D600060215502031D0800683062020319282F04
:101D700025166C30620203199C2F6D306202031924
:101D8000BB2F3230620203195F2F44306202031D01
:101D9000080016308A00D7260E308A000800D001CD
:101DA000D1011430B100B00146302F117B242B0833
:101DB000D0002C08D1000800E001E1010800A801D2
:101DC000A901AA01523084005624543084005624BC
:101DD0005630840056245830840056244F0864241A
:101DE0005E3084005624B0015F081A3C031CFB2EB1
:101DF0005F08B100FD2E1A30B1005A3084002F1553
:101E00007F242909E0002809E100080044305D0230
:101E1000031D102F15308A0076250F308A00080028
:101E200007305D02031D08001723E5250A25DC267F
:101E3000CF26C4245A08A7005C08DA002708DC0073
:101E40005B08A7005D08DB002708DD0038230800D9
:101E50003727142F6830E20037271A30DF00DE0101
:101E6000B2010D308A00FA250F308A0008000130D7
:101E7000E3002330E40008002F1637180800370865
:101E8000B1003608B0003C30B102031CB0032F1281
:101E900008002F16311C502F01301022A700532F9D
:101EA00000301022A7000130B10203185C2F01306E
:101EB000B002031C08005C2F2F12270808003C27E3
:101EC0002F1A0800A030B20049272F1A942F0000C3
:101ED0006430270203190121773027020319892F63
:101EE000733027020319A021613027020319E22170
:101EF0006E3027020319DF21703027020319AC214D
:101F000072302702031D642F32088400C221B20AF6
:101F1000642F49272F1A08002708A1002108A700CD
:101F200027308400D521642FA030B2021A30DF00A0
:101F3000DE013208DF07FA2D3C272F1A0800023095
:101F4000B1020318A72F0130B002031C08000030B3
:101F50001022A700023027020319B32F03302702F3
:101F60000319B72F08000130102276209F2F01306F
:101F7000102284209F2F18308A000E200F308A00F4
:101F80003C272F1A0800B108031DC92FB0080319F8
:101F9000F82F18308A0009200F308A0000308500A1
:101FA0000918CC23B0080319DD2FFE30E2270230D8
:101FB000B1070318D02FB003D02F0918CC23310854
:101FC000E227F82F831686018312860007178717EA
:101FD00087130713831686030514081783128914C1
:101FE0000919F02F831605100813831289100800B1
:101FF00018308A002C200F308A000918CC230800E2
:10200000031714080313080008308A0092201030C8
:102010008A000800BC00BB003F3084003E213E2106
:102020003E213E210B30BD00BE1CBD0108308A00A0
:102030000E30762010308A003E1008308A00C03002
:10204000762010308A000321F0200B308A00A6236E
:1020500010308A0000206E3C0319BE2800205F3C2F
:102060000319BE2800202B3C0319BE2800202B3C5E
:102070000319BE2800200E3C0319BD2800203F3C58
:102080000319BD2800200B3C0319492800201F3CE0
:102090000319C72000208B3C0319512800204F3C16
:1020A0000319D02000204B3C0319592800206F3C15
:1020B0000319D9200020CB3C0319612800202F3CB4
:1020C0000319DB20CD010020763C03196A2800208B
:1020D000673C0319E6200020863C03197228002083
:1020E0000F3C0319E5200020463C03197A28002004
:1020F000F73C0319E4200020C63C03198228002085
:10210000773C0319E3200020263C03198A2800208D
:10211000B73C0319E2200020A63C031992280020B6
:10212000373C0319E1200020663C03199A2800205F
:10213000D73C0319E0200020E63C0319A228002028
:10214000573C0319DF200020163C0319AA28002061
:10215000973C0319DE200020963C0319B22800208A
:10216000173C0319DD20BE013D080C3C0319BE28B5
:102170003D0F1C28BD283E140800BE143F308400CB
:102180003C08BB005D215D215D215D2108003D080B
:102190003F3E8400800A00080A3C031980000800C2
:1021A0003D083F3E84008003000F08000930800096
:1021B0000800BD030800BD0A0800CD0ACD0ACD0AFB
:1021C000CD0ACD0ACD0ACD0ACD0ACD0A3D083F3E43
:1021D00084004D0880003D080B3C031DDB200800F7
:1021E0003D08A0000C308A0003304B2410308A00D8
:1021F0003D082207C13EA30008308A00230876204C
:1022000011308A0008003F30840008308A005B30BB
:10221000842011308A00282108308A002E30842042
:1022200011308A00282108308A002E308420113095
:102230008A00282108308A002E30842011308A003C
:10224000282108308A005D30842011308A0008007F
:1022500008308A000008D22011308A00840A083031
:102260008A000008D22011308A00840A08308A00CF
:102270000008D22011308A00840A080009308A0040
:102280003B08602111308A002308A0000C308A002E
:1022900064304B2411308A0022088000840A0C30FC
:1022A0008A000A304B2411308A0022088000840AF8
:1022B00020088000840ABB0A0800A1010008031955
:1022C000652980036430A1075E29840A0008031988
:1022D0006D2980030A30A1076629840A0008A10736
:1022E0003B08A00009308A006B2111308A00840A63
:1022F000BB0A080008308A00922011308A000800CA
:10230000BE017A211630BB0009308A003B086021EB
:1023100011308A002308031D04280630AD009430D4
:10232000AE0008308A00B12011308A0009308A00DE
:10233000042111308A007A210630AD00B830AE0099
:1023400008308A00B12011308A000630AD00CB3051
:10235000AE0008308A00B12011308A000B308A00AC
:10236000A62311308A0000200B3C0319F429002019
:102370001F3C0319F42900208B3C0319F429002089
:102380004F3C0319F4290020CB3C03192B2A0020D1
:102390002F3C03192B2A00206E3C03192B2A002006
:1023A0005F3C03192B2A00202B3C03192B2A002009
:1023B0002B3C03192B2A0020003C03192B2A002058
:1023C000003C03192B2A7A210630AD00F730AE000D
:1023D00008308A00B12011308A0009308A000421B7
:1023E00011308A007A219B290630AD00E130AE0021
:1023F00008308A00B12011308A000B308A00A623F1
:1024000012308A0000200B3C0319A52900201F3C34
:102410000319A52900208B3C0319A52900204F3C56
:102420000319A5290020CB3C0319362A00202F3C94
:102430000319362A00206E3C0319362A00205F3C1F
:102440000319362A00202B3C0319362A00202B3C86
:102450000319362AF4297A210730AD007630AE0010
:1024600008308A00B12012308A0004284C10CC10A9
:10247000031715308D0009308A00622112308A005E
:1024800000302302031D4C14023023020319CC1424
:102490001530A0007A210730AD002030AE000830A2
:1024A0008A00B12012308A00BE104C1CC82ACC1CF5
:1024B000912A0730AD003430AE0008308A00B120D8
:1024C00012308A0000000B308A00A62312308A00E6
:1024D00000200B3C0319C82A00201F3C0319C82AFE
:1024E00000208B3C0319912A00204F3C0319912AAC
:1024F0000020CB3C0319132B00202F3C0319132B76
:1025000000206E3C0319132B00205F3C0319132B92
:1025100000202B3C0319132B00202B3C0319132BF9
:10252000592A0730AD004A30AE0008308A00B12089
:1025300012308A000B308A00A62312308A00002055
:102540000B3C0319592A00201F3C0319592A00206B
:102550008B3C0319C82A00204F3C0319C82A0020CD
:10256000CB3C0319092B00202F3C0319092B002019
:102570006E3C0319092B00205F3C0319092B002036
:102580002B3C0319092B00202B3C0319092B912A02
:102590000730AD006030AE0008308A00B120123044
:1025A0008A000B308A00A62312308A0000200B3CE0
:1025B0000319912A00201F3C0319912A00208B3C0B
:1025C0000319592A00204F3C0319592A0020CB3CFB
:1025D0000319FF2A00202F3C0319FF2A00206E3C1C
:1025E0000319FF2A00205F3C0319FF2A00202B3C1F
:1025F0000319FF2A00202B3C0319FF2AC82A4C107C
:10260000CC100030A10009308A006B2113308A0001
:102610001D2B4C14CC100130A10009308A006B2115
:1026200013308A004D2B4C14CC140230A100093019
:102630008A006B2113308A00602B7A210730AD00AD
:102640008830AE0008308A00B12013308A00003094
:102650000A203E18362ABE18362A7A210730AD00E5
:102660009B30AE0008308A00B12013308A0004305D
:102670000A203E18362ABE181D2B7A210730AD00DD
:10268000AE30AE0008308A00B12013308A000C3022
:102690000A203E18362ABE182D2B7A210730AD00AD
:1026A000C230AE0008308A00B12013308A000830F2
:1026B0000A203E18362ABE1C602B4C1C3D2B362AA5
:1026C0007A210730AD00D230AE0008308A00B12048
:1026D00013308A000B308A00A62313308A000020B2
:1026E0004B3C0319982B00206F3C0319982B0020BA
:1026F0000E3C0319982B00203F3C0319982B002017
:10270000CB3C0319042800202F3C03190428002087
:102710006E3C0319042800205F3C031904280020A4
:102720002B3C0319042800202B3C031904286A2B96
:10273000CC1C4D2B362A25160B308A00172313305C
:102740008A0003305A0203190B2C08305A02031D69
:10275000572C08308A000230762013308A00063069
:10276000AD004130AE0008308A00B12013308A003D
:102770005A08A10008308A00622013308A0006300F
:10278000AD004730AE0008308A00B12013308A0017
:102790006108A10008308A00622013308A006008B6
:1027A000A10008308A00622013308A000630AD0094
:1027B0004F30AE0008308A00B12013308A00143048
:1027C0008A00252413308A00DC01DD01DA01DB01F7
:1027D0000D308A00E52513308A000D308A000A2565
:1027E00013308A000E308A00CF2613308A001A3048
:1027F000B100B0012F150C308A005A307B24133001
:102800008A002B08DC002C08DD000B308A003823FE
:1028100014308A00572C08308A0002307620143099
:102820008A000630AD005430AE0008308A00B12076
:1028300014308A0025240630AD007530AE00083013
:102840008A00B12014308A00572C00005208A000E2
:1028500008308A00D52014308A0008308A002E30D3
:10286000842014308A005308A00008308A00D52044
:1028700014308A0008308A002E30842014308A00F8
:102880005408A00008308A00D52014308A0008308F
:102890008A002E30842014308A005508A0000830A9
:1028A0008A00D52014308A0013308A0008000A30CC
:1028B0008A000800831203130800013083160317EF
:1028C0009A00831203130E0883160317A0008312C5
:1028D00003130F08831603179F00831203130800C6
:1028E0008316031701301A020319192D02301A0238
:1028F0000319382D5A2C0B308A00872314308A0094
:102900000800AB01AC01A000A00C0B308A008723AB
:1029100014308A00A00B852C08000B308A0093230A
:1029200014308A002C08080003178D0009308A0033
:10293000622114308A0023080800A200A2080319AB
:1029400008008D24A20BA12C080011308A007A21E6
:1029500014308A000630AD007730AE0008308A00AF
:10296000B12014308A000C308A00B12414308A005F
:102970000D308A00292514308A00FF30D600D70098
:10298000D800D900D201D301D401D501DA014430F5
:10299000DB00DC014330DD000230DE002C30DF00E4
:1029A0000130E2000130E3000630E400E5010130CF
:1029B000E6000230E700831603171F088312031393
:1029C000E80083160317200883120313E900EB01C4
:1029D0000230EA000030EC00ED01EE01EF01F00101
:1029E000F101F201F301B2010E308A002E261430FB
:1029F0008A00AB01AC010A3081243E08AB003F08DD
:102A0000AC007B244008AB004108AC007B244208AA
:102A1000AB004308AC007B24CA3081246330AB0098
:102A20008230AC007B245330AB006330AC007B249D
:102A3000080083120313A5243530AB000130AC002D
:102A40007B240130AB00AC017B243330AB0004307D
:102A5000AC007B24FF30AB00AC007B247B24FF3038
:102A6000AB00AC017B24FE3081242A308124080095
:102A700083120313A5243530AB000130AC007B2456
:102A80000330AB00AC017B243630AB000430AC002B
:102A90007B2483179B3084000008AB00840A000865
:102AA000AC007B24840A0008AB00840A0008AC0058
:102AB0007B2483133230AB000430AC007B24003025
:102AC0009424AB0001309424AC007B240230942485
:102AD000AB0003309424AC007B24FF30AB00AC018E
:102AE0007B24FE30812424308124080002306202DD
:102AF000031D5A2C01306602031D5A2C0230670256
:102B0000031D5A2C831603171F0883120313680230
:102B1000031D5A2C8316031720088312031369021E
:102B2000031D5A2C8316031701301A0203199D2D19
:102B30008312031302309D24C02D8312031300302F
:102B4000A0007208A10009308A006B2115308A00AC
:102B5000A00A7308A10009308A006B2115308A0091
:102B6000A00A8D24A10009308A006B2115308A004B
:102B7000A00A8D24A10009308A006B2115308A003B
:102B8000D8309D2404309D248D240319C42DFF309A
:102B90002C0203193D2E01302C020319DE2D0330C7
:102BA0002C020319012E35302C020319282E363041
:102BB0002C020319302E8D249D24C42D8D248D24A8
:102BC000A1000430A00009308A006B2115308A0072
:102BD0008D24A100A00A09308A006B2115308A00DB
:102BE0008D24A100A00A09308A006B2115308A00CB
:102BF0008D24A100A00A09308A006B2115308A00BB
:102C0000C42D8D24043CB1008D24A1000C30A00003
:102C100009308A006B2116308A008D24A100A00A99
:102C200009308A006B2116308A008D24A100A00A89
:102C300009308A006B2116308A008D24A100A00A79
:102C400009308A006B2116308A0031089D24C42D7A
:102C50008D248D2483160317990083120313C42D2A
:102C60008D249B3084000430A3008D2483178000C2
:102C70008313840AA30B352EC42D83160317023049
:102C8000190203194E2E053019020319542E05306E
:102C9000190203195A2E83120313080002309A00F6
:102CA00083120313A515080004309A00831203133E
:102CB0002514080001309A0083120313A51508009B
:102CC000A51F692E08308A000130762016308A0050
:102CD000A513251F080025130800A511031715309B
:102CE0008D0009308A00622116308A0001302302EB
:102CF0000319A51400302302031D802EA5142514EA
:102D00002518882E14308A00702416308A00080096
:102D1000A5188B2E9D2E2519942E03172430900074
:102D200003130D308A00312D83120317900B9B2E55
:102D3000031325118B2E0313080011308A007A210A
:102D400016308A000630AD008630AE0008308A00AA
:102D5000B12016308A000C308A00B12416308A0067
:102D60000D308A00292516308A000D308A00ED25A5
:102D700016308A00FF30D600D700D800D9000D30B9
:102D8000DA009B30DB000D30DC009B30DD00DE0123
:102D90001A30DF006430E2000130E4001130E50059
:102DA000B2010E308A002E2616308A000800E40890
:102DB0000319E62E6408D2006508D3006608D40023
:102DC0006708D5006808DA006908DB000830A00051
:102DD0005208A10009308A006B2116308A00A00A2F
:102DE0005308A10009308A006B2116308A00A00A1E
:102DF0005408A10009308A006B2116308A00A00A0D
:102E00005508A10009308A006B2117308A00123062
:102E1000A0005A08A10009308A006B2117308A00EF
:102E2000A00A5B08A10009308A006B2117308A00D4
:102E3000A51408000317E3308D0009308A006221D1
:102E400017308A00A30A031D0800E330A0000830F1
:102E50008A000320A10017308A0009308A006B2104
:102E600017308A00A00A08308A000220A10017301B
:102E70008A0009308A006B2117308A00A00A0830C6
:102E80008A000120A10017308A0009308A006B21D6
:102E900017308A00080001309B0060309C00080059
:102EA00003171119542FB22F0313251603170230DD
:102EB0001402031D672FF7301502031D672F003022
:102EC0001602031D672F003017020319B42FBF30FD
:102ED0001402031D772F40301502031D772F893010
:102EE0001602031D772F763017020319B42F4B27D4
:102EF00003136930E200E3018316031713088312FA
:102F00000313E40083160317140883120313E50068
:102F10000F08E6000E08E70003171A080313E8007D
:102F2000031713080313E900031717080313EA0034
:102F3000031716080313EB00031715080313EC001F
:102F4000031714080313ED00DE011A30DF00B2018D
:102F50000D308A00FA2517308A000B308A009E2334
:102F600017308A00031308009C0B782F9B0B782FD7
:102F7000031308308A00922017308A000730AD0012
:102F8000EF30AE0008308A00B12017308A000930D7
:0E2F90008A0001300B2117308A00AF17B22FD4
:10300000831203130800492083160317A501251412
:10301000002868088620690877200800E3185420F3
:10302000631825281E28B7205F206A2083160317FF
:103030002518002883120313C520080083160317E0
:10304000251083120313C5200800831603172514C7
:1030500083120313B720080083120313132083166F
:103060000317230883120313EA00831603172408A7
:1030700083120313EB00831203136130E2001A3052
:10308000DF00DE01B2010D308A00FA2518308A0017
:10309000002883160712871207138711871307105A
:1030A0000914891009158312071287120713871153
:1030B00089108713071407100714B7200800871515
:1030C000871706088713871183160317A300831237
:1030D000031308008715071687170608871387113B
:1030E000071283160317A400831203130800831624
:1030F00086018312871607168600871787138316A3
:103100008601860383128712071208008316860140
:103110008312871686008717871383168601860316
:1031200083128712080087158716871706088713EA
:10313000871187120800831686018603831287157C
:1031400087160716000087170608A20087130000DD
:1031500087118712071208008316860183128600E2
:103160008717871383168601860383120800831648
:10317000860183120716003086008717871383168F
:1031800086018603831207120800831686018312C4
:10319000071601308600871787138316860186037A
:0631A00083120712080073
:02400E00723FFF
:104200000A0000000100DF00FF00FF00FF000000C7
:104210000A0000000100CC000A00000001000100BB
:0E4220000D009B000D009B000200020000003C
:0C43C000000004002000FF0000000000CE
:00000001FF
